:020000020000FC
:10000000A6CDAEC10000000020C000008EC00000E0
:10001000000098C000000000000000000203040679
:10002000080C10182030406080000406080C1018DE
:100030002030406080A0C0000003070F1F000D0D9E
:1000400004050D050305030302004FB662FD0CC055
:10005000552041F00994C52DC095089483FDC7959E
:10006000C4BD64604FBE1895C0916400089483FDC0
:10007000C795C4BD6B7FC0916400CF3F09F41EC01B
:1000800070FF1AC082FD05C04FBE9598AC98C0980D
:10009000189576FD0EC065FD0CC0C091B100C0FD85
:1000A0009498C1FDAD98C2FDAB98CAEFC095CA95B2
:1000B000F1F79598AC98C0984FBE189524BCCC2702
:1000C000C064C8BF6460F8CFC6CF70FFC4CF65FD01
:1000D000C2CF959AC0CF70FFBECF65FDBCCFAC9AA2
:1000E000BACF70FFB8CF65FDB6CFC09AB4CF949A9F
:1000F00070FFB1CF65FDAFCFC7E0CA95F1F7959A14
:10010000AACFAD9A70FFA7CF65FDA5CFC7E0CA956E
:10011000F1F7AC9AA0CFAB9A70FF9DCF65FD9BCF56
:10012000C7E0CA95F1F7C09A96CF4FB6C9B7CF7E50
:10013000C9BF6E7FCCB5CE0DDDB5DF1DDBBDCABD41
:100140004FBE18953FB68F7EABB7A074A2118061E9
:10015000A0E0ABBFA9B7AE7FA9BF7894A09168001B
:10016000AA2341F085FD2AC0A0916800AA95A0931A
:10017000680024C040E050E085FD14C0A0B396FDA7
:10018000A095A2FD4FEFA3E096FDA2E0A5BFAA2790
:10019000A064AABF8D7FA0B396FDA095A2FD5FEFDE
:1001A000451741F7A8E161FDA093680085FD03C0F4
:1001B000A8E1A093680040939600816085FD0EC081
:1001C000A0916900AA2331F0A0916900AA95A0939B
:1001D000690004C08061AA27A064AABF80FF3CC058
:1001E000A09196004A2F61FF8E7F85FD1CC0A091D3
:1001F000B400A430C1F4403F08F040EFA42FA29512
:10020000AF704A0F5091B600533069F0A695A6958D
:1002100050FD01C0A69552FD03C0A41B4A2F03C088
:100220004A0F08F44FEF40936100A72FA670A1F08A
:1002300073FD12C0A0917000AA0FAA0F50919E00EA
:1002400056955695541708F0452F4A0F4093610074
:1002500018F4AFEFA09361004091B400443009F06E
:100260003EC0A0916100A093630040916300A09103
:100270009B004A1708F04A2FA0919D004A1708F0EA
:100280004A2F542EA091A000AA2309F422C0542F73
:100290005A1B10F4A42F50E0BA2E8894AA1FAA2E3D
:1002A000A091A200A095AA22A50E58F0A091A100AD
:1002B000A21509F0AA95AA0EA093A10048F04A2D14
:1002C00008C0A091A100BA1608F0A395A093A100C0
:1002D0004FEF409364007F7B485F08F07064A52D6A
:1002E000A03408F06860A0916000A395A09360001E
:1002F00051F0F894A9B7A160A9BF84FF02C0A0E49F
:10030000ABBF3FBE1895A0917400A395A093740055
:1003100041E050916800552329F085FF03C05A95AC
:1003200050936800A0919600A13018F02092990097
:100330000DC020929A002092A300A0919900AF5F77
:10034000A093990018F0AFEFA0939900F894A9B783
:10035000A160A9BF84FF02C0A0E4ABBF3FBE189557
:100360003FB64CB55DB58F7EABB7A074A21180616E
:10037000A0E0ABBFA9B7AE7FA9BF789481FD23C031
:10038000A2E096FDA3E0A5BF8260A0B396FDA09574
:10039000A2FF05C040936500509366003EC1A3E0F4
:1003A00096FDA2E0A5BFAA27A064AABF8D7F85FF06
:1003B00001C026C140E0A0B396FDA095A2FD20C1DA
:1003C000409396000FC1A3E096FDA2E0A5BF8D7FEC
:1003D00061FF71C0A2E096FDA3E0A5BFAA27A064BB
:1003E000AABF82604093910050939200A0908F002A
:1003F0004A19B09090005B09BB24A22C4C385205DE
:1004000018F42092950049C0A091D400AA2359F174
:10041000483C520528F4A0E1BA2EAAE0AA2E23C037
:100420004836A1E05A0728F4A8E0BA2EAFE0AA2E79
:100430001AC0403DA2E05A0728F4A4E0BA2EAEE16B
:10044000AA2E11C0403AA5E05A0728F4A2E0BA2E1D
:10045000ACE3AA2E08C04839A8E05A0720F4A1E06E
:10046000BA2EA8E7AA2EC42EA0919300CA1AD52EA0
:10047000A0919400DA0ADD202AF4AFEFC094D09462
:10048000CA1ADA0A20929500A8E0A210A0E0CA14C5
:10049000DA0618F4A1E0A0939500409393005093DE
:1004A0009400409191005091920040938F0050939E
:1004B000900042E097C0A09165004A1BA0916600A1
:1004C0005A0B94FD82C093FD80C092FD7CC086FFD4
:1004D00003C0D52EC42E0CC05695479591FD73C010
:1004E0005695479590FD6FC0D52EC42ED694C794CF
:1004F00061FD19C0AC2DAC51AD2DA24008F005C076
:10050000DD2089F4AC2DA85C70F4A0916700A39560
:10051000AA2311F0A0936700AA3008F471C02092BA
:10052000960081606DC0A0916700AA2319F0AA957A
:10053000A0936700A22C5091BA0097FD06C0A0902E
:10054000C800533011F4A090D000AAEFAA0EA22D3B
:10055000A21DCA18DA0A4FB74170533049F4442338
:1005600021F087FD05C0806803C087FF01C08F7739
:10057000442359F0533031F4AFEFC094D094CA1AE9
:10058000DA0A03C040E050E020C0533049F4CC0CFC
:10059000DD1CAAE0CA1AD20818F4A0E0CA2ED22C98
:1005A000AFEFCA16D20418F04FEF50E00EC0A09182
:1005B000AC00CA9E412D000C441F50E008F012C050
:1005C0004FEF50E00FC05695479594FF07C0552355
:1005D00009F04FEFA42FA6954A0F521D4F3F520529
:1005E00008F04FEF40939600816061FF09C0AFE1D2
:1005F000A095A923AB299A2F8F7DBB2009F4806297
:10060000A8E1A093680085FF03C0AAE0A09368005A
:1006100061FD03C085FD01C08F7E85FD03C0A6E09E
:10062000A0936900F894A9B7A160A9BF84FF02C094
:10063000A0E4ABBF3FBE189511E00AC013E008C0AC
:100640001AE006C01EE104C014E602C018EC00C0A7
:1006500005E1BB27BA95F1F70A95D9F71A95C1F7C5
:1006600008952AE338E709C020E33CE806C02AE2FF
:1006700034EB03C025E238EC00C012E0BB27AD9A92
:10068000BA95F1F7AC9ABA95F1F7AC98BA95F1F73B
:10069000AD98BA95F1F7123009F0959A123009F435
:1006A000C09AB091AD00BA95F1F7123009F0959863
:1006B000123009F4C098B7E8BA95F1F71A95F1F637
:1006C000022FB22FBA95F1F70A95D9F73A95A9F604
:1006D000AD9A0895221B39E0001F3A9509F4089558
:1006E000221F211B18F4210F8894F6CF0894F4CF11
:1006F000622C722CB0E08894B395221F331FE0F770
:10070000379527958894912E802E020B130B10F4A9
:10071000192D082D10F4889401C00894661C771CCC
:10072000BA9571F7172D062D0895322D11232AF44D
:100730003A9500951095031B130BF894029F712CAA
:10074000002D129F912C802C7894780C172D921CE0
:10075000292DB4E06B2E2695179507956A94D9F745
:10076000332321F000951095031B130B089500917E
:10077000B4000430A1F1B0919600B15008F010C05F
:10078000B0916100B093630020927E0020927F00C0
:100790002092800020928100209282006F7B1FC0F7
:1007A0006090B4006064B0916100B093620008E3AF
:1007B00017EC20917A0030917B0036952795B62D65
:1007C000BA9541F036952795B62DBA95BA9511F0A0
:1007D000369527958DDF00937E0010937F00089556
:1007E00000917E00B09162000B1B10917F001209F6
:1007F00028F40038BFEF1B0740F009C00F3712057F
:1008000008F405C00FE710E002C000E81FEF0093F6
:10081000830010938400089500918300B0918000BC
:100820000B0F10918400B09181001B1F20E03091CC
:10083000840033230AF42A95B09182002B1F1AF406
:10084000203F40F00AC02F3008F407C00FEF1FEF21
:100850002FE003C000E010E020EF30916300B09182
:100860009B003B1718F4323030F009C0B09184007F
:10087000BB235AF004C0B0918400BB2332F4009330
:100880008000109381002093820008952091D7006A
:1008900000918300000F10918400111F46DF112387
:1008A0002AF40038BFEF1B0740F009C00F371205CC
:1008B00008F405C00FE710E002C000E81FEF0023B6
:1008C00052F0B0916200B01B0B2F18F0013008F00D
:1008D0000AC001E008C000950F5FB09162000B0FE5
:1008E00008F001C00FEF0093850008952091D80013
:1008F000009181001091820018DF11232AF4013049
:10090000BFEF1B0740F009C00F3F120508F405C0F8
:100910000FEF10E002C001E01FEF112352F0B09181
:100920008500B01B0B2F18F0013008F00AC001E061
:1009300008C000950F5FB09185000B0F08F001C053
:100940000FEF0093630008950FEF677F71FD29C0DB
:1009500072FD09C06860B0917B00BA3020F0B52DFF
:10096000B03408F4677FB091D300BB23D1F0B091CD
:100970007B00BB23B1F00FEF10917B00ABDEF8944E
:10098000B091730072FDB5E00B9F112D002D78948E
:10099000112309F00FEFB0919E000B1710F4009196
:1009A0009E0000939D00089500917A0010917B00B5
:1009B00000541140B0919D0010F4BA9501C0B39558
:1009C00011F0B0939D00089500C008952091B500E6
:1009D000B6B1B6FDFBCF04B115B1B6B1BF77B6B9AC
:1009E000B091AA00B395B093AA00B83060F12092FC
:1009F000AA00B091D200BB2321F1112329F0B091BC
:100A0000AB00BF3F61F009C0B091AB000B1739F0EC
:100A100020F4BB2321F0BA9502C0B395E1F3009115
:100A20009B00B093AB00B83850F400ECBD3738F4FD
:100A300000E8B23720F400E4B73608F400E0009391
:100A40009B007F7E089510919B00B0E11B0F08F47E
:100A50001FEF10939B00B091B400B43081F000916F
:100A60009B00B0916300B01B10F400916300B09143
:100A70009D000B1708F00B2F502E00936400B091CF
:100A8000AA00B73009F47061089502E3F894B091B8
:100A9000D9000B9F012D000C001F7894B0919B0092
:100AA0000B1710F000919B0000936100009363000E
:100AB000502E0093640000939E00089520927A00C7
:100AC000B0EFB0937B000895F8940CB51DB520915C
:100AD00074007894309175006090760000937500F2
:100AE00010937600031B160971FD03C077FD7DC0CE
:100AF00027C070907700209377002709222311F0F8
:100B00000FEF1FEF8090780090907900309378007D
:100B1000609279000091750010917600081919090A
:100B200020917A0030917B0036952795020F131F94
:100B300010F40FEF1FEF00937A0010937B0029C091
:100B400020917A0030917B003901B4E08B2EB2E025
:100B50009B2E343010F08A949A94383010F08A9496
:100B60009A94769467948A94E1F726193709992024
:100B700021F0169507959A94E1F7200F311F2093E5
:100B80007A0030937B0028F43FEF30937A00309363
:100B90007B00323008F4706871FF02C0B3E00DC012
:100BA000B091C40000917100023838F0B395003A5A
:100BB00008F0B395B63008F0B5E09B2EB4E08B2E6C
:100BC00010917B0000917A0024E0169507952A95F4
:100BD000E1F70819120928F0B02FB250B12FB2096D
:100BE00010F402E010E0980126C020917A003091C4
:100BF0007B0039017694679466946694669426190E
:100C0000320906950695200F321D20937A00309305
:100C10007B00323008F07F7704E0369527953695D3
:100C2000279526952695201B10F0223008F422E007
:100C300089019090C40060FDFECFE0908B00F090A1
:100C40008C006160B9B7B061B9BF380177FD41C0B0
:100C50007694679400938B0010938C00B92DB33079
:100C6000E1F0B0FD04C0060D171D930106C0000F92
:100C7000111F0250120922E030E0B92DB33068F0A4
:100C800020938D0030938E0000938700109388008E
:100C90006092890070928A003AC000938D00109390
:100CA0008E002093870030938800609289007092B4
:100CB0008A0071FF0DC0BFE0B0938D0020928E00BE
:100CC000B093890020928A00B0938B0020928C0010
:100CD0001EC0669400938B00B92DB33091F0B0FD27
:100CE00003C0060D262D03C0000F025022E0B92DCF
:100CF000B33038F020938D00009387006092890014
:100D000006C000938D0020938700609289000091B7
:100D10007C0002FD0350013029F495FD0AC0B6E0C5
:100D2000B7B909C0023019F4B7E0B7B904C095FDEE
:100D3000F6CFB0E0B7B90091A200000F10F4BBE607
:100D40000B270093A20060FDFECFB2E0B0936E00CF
:100D50006160B9B7B061B9BFB72FB670D1F020915B
:100D60007A0030917B00369527953695279571FF4F
:100D700002C0B0E43B0FF8940CB51DB5020F131F71
:100D80001BBD0ABD6160B0E1B8BFB9B7B061B9BF02
:100D900078940895606120927D0020E067FD20E254
:100DA00006C0606120927D0020E267FD20E001E046
:100DB00011E077FD11C0B72FB67009F06F7E14E116
:100DC00000917B00069509F403950F3008F00FE0C1
:100DD00071FF02C004E114E160FD0FC0B0917D001D
:100DE000BB2359F071FF06C0B0916E00BA95B09365
:100DF0006E0011F4706247C0ABDFB0B7B77FB0BF11
:100E0000B8B1B0B7B860B0BFB0917D00B395B09342
:100E10007D00B8B177FD06C0B1E071FDB3E0BA95D1
:100E2000F1F7B8B1B072B21709F022C071FF05C076
:100E30000395011708F00A95CFCF64FD05C003950F
:100E4000011708F0B4CFC8CF6F7EF8943CB56DB4ED
:100E500070907A0080907B00370D681C6BBC3ABDA7
:100E60006160B0E1B8BFB9B7B061B9BF78949FCF46
:100E7000B0916D00B13008F49ACF64FD98CF0A9517
:100E800009F0AACF7F7D20918D0030918E00F894DB
:100E9000B0E1B8BF0CB51DB5020F131F1BBD0ABDD5
:100EA000E0908700F09088006160B9B7B061B9BF89
:100EB0007894B72FB67039F0B0916D0072FFB3958A
:100EC000B0936D0009C075FF07C067FD05C064FDE4
:100ED00003C0BF91BF91EBC4089500E063FF03C05E
:100EE00064FF01C001E0F89410917100B7E01B9F0E
:100EF000212D102D7894200F26951795269517955E
:100F00002695179510937100183718F4B8E7B09329
:100F1000710000917100B09172000B1720F06062B7
:100F20009598AC98C09860FDFECFE0908900F09055
:100F30008A006160B9B7B061B9BF0895B2E095FDAC
:100F40000AC0F894B0937C00AD9A949862FF01C0F7
:100F5000C09A7894F4C0F894B0937C00AD9AAB98A2
:100F600062FF01C0959A7894EAC0B3E082FF24C082
:100F700095FD11C002E0F894B0937C00E1E8F0E048
:100F80000093B100C098AB9A62FF02C0AC9A01C056
:100F9000AD987894D4C002E0F894B0937C00E1E876
:100FA000F0E00093B1009598949A62FF02C0AC9A69
:100FB00001C0AD987894C3C095FD0BC0F894B09370
:100FC0007C00EBE6F0E0C09862FF01C0AC9A789438
:100FD000B6C0F894B0937C00EBE6F0E0959862FF21
:100FE00001C0AC9A7894ABC0B4E095FD0AC0F89407
:100FF000B0937C00949AAB9862FF01C0AC9A78944D
:101000009EC0F894B0937C00AB9A949862FF01C0A4
:10101000AC9A789494C0B5E082FF24C095FD11C0CD
:1010200001E0F894B0937C00E7E7F0E00093B100B2
:10103000AC98AD9A62FF02C0959A01C094987894DA
:101040007EC004E0F894B0937C00EBE8F0E00093FD
:10105000B100AC98AD9A62FF02C0C09A01C0AB98D3
:1010600078946DC095FD0BC0F894B0937C00E5E6D4
:10107000F0E0AC9862FF01C0959A789460C0F89453
:10108000B0937C00E1E7F0E0AC9862FF01C0C09A49
:10109000789455C0B6E095FD0AC0F894B0937C00F2
:1010A000AB9AAD9862FF01C0959A789448C0F894C5
:1010B000B0937C00949AAD9862FF01C0C09A789476
:1010C0003EC0B1E082FF24C095FD11C004E0F89459
:1010D000B0937C00EBE8F0E00093B1009598949A0F
:1010E00062FF02C0C09A01C0AB98789428C001E0AA
:1010F000F894B0937C00E7E7F0E00093B100C0986B
:10110000AB9A62FF02C0959A01C09498789417C078
:1011100095FD0BC0F894B0937C00E1E7F0E0959862
:1011200062FF01C0C09A78940AC0F894B0937C0022
:10113000E5E6F0E0C09862FF01C0959A78946F7D73
:10114000089524E630E0F9012092B1009598AC981A
:10115000C098949AAD9AAB9A6B7F0895A2EBB0E0D9
:1011600009E00D9309E00D9304E00D930FEF0D934B
:1011700003E00D930FEF0D930BE00D9303E00D9340
:1011800001E00D9301E00D93AEEBB0E001E00D93B3
:101190000FEF0D930D930D930D930D9303E00D93AE
:1011A0000FEF0D930FEF0D930D9305E20D9300EDEF
:1011B0000D9308E20D9300E50D9304E00D930FEFFE
:1011C0000D9302E00D9300E00D930AE70D930FEFEE
:1011D0000D9300E00D9301E00D9300E00D9303E00B
:1011E0000D9300E00D9308952091B9008B7F23307B
:1011F00009F48460B091BA00B33019F09F7DB1FD5D
:1012000090629F7BB091BB00B1FD9064223011F0E1
:10121000886001C0877F08950A95E00FF21DB491A0
:101220000895ECE1F0E00091B200F6DFB093D70052
:10123000ECE1F0E00091B300EFDFB093D800EAE218
:10124000F0E00091B800E8DFB093D9000091B80059
:10125000023008F402E000937300B091CE000FEF6B
:10126000B23009F400EAB33009F402E800937200E6
:10127000E8E3F0E00091D500CFDFB093A00008953F
:1012800008952091C8003091C900B091BA00B330E0
:1012900009F43E5097FF02C020E03FEFB32FB21B8E
:1012A0006B2EB25810F4B2E86B2E00E00395609EEE
:1012B000B12DBD57D8F30093AC0008959068E1DFDD
:1012C000C1D920E030E0B0E16B2EB8D9B0919600E2
:1012D0002B0F321D6A94C9F7B4E036952795BA955D
:1012E000E1F7822E9F77CDDF0895F894E3E0F0E0F8
:1012F000B9E0B7BFB491B078C1F3F894A895B1B58F
:10130000B861B1BDB0E0B1BDB4E0BEBFBFE5BDBF27
:1013100018DFB0E0B8BBB1E1B7BBB8E2B5BBB8E32A
:10132000B4BBB0E1B2BBB0E3B1BB2224A0E0B0E0FB
:101330002D92AA31E9F7A0E6B0E00FEF2D920A95C1
:10134000E9F7B1E0B093A20009DFE9D2B6B1B46029
:10135000B6B90091CA000093AD00B1E0B0936A0045
:10136000F89474D97ED96ED97FD96CD980D96AD9CD
:10137000F8940AEF1AEFA0B396FDA095A2FF1FC044
:101380001A95C9F70A95B1F7E0E0FCE1B591B43ED2
:1013900039F4B591B03E21F4B591BF3F09F40CC0CA
:1013A000E0E0F395F395B591B83F49F4B591B439C0
:1013B00031F4B591BA3A19F4EE27F695099414DF91
:1013C00030DF5EDF5EDF0091CA000093AD00B9DE62
:1013D000B2E0B3BFB2E0BEBDB2E0B5BDB1E5B8BFEB
:1013E000B9BFB0B7B77FB0BFB8B1B0B7B860B0BF22
:1013F00023D97894E9DA20927000B3E096FDB2E048
:10140000B5BFB0E4BBBFBB27B064BABF8D7F1ED9E8
:10141000626033E02CE0B0919500BB2321F42CE016
:101420003A9509F4A5CF0ED980FFA2CF8E7FB09157
:101430009600B23078F3B92FBF71009198000093F5
:101440009700B0939800B01729F72A9521F76D7F80
:10145000B3E096FDB2E0B5BFBB27B064BABF8D7FE5
:10146000B091D400BB2321F48062B92FB0709B2FC0
:101470008F7B20926700E8D885FF05C0B091670098
:10148000BA3008F08064DAD802E085FF01C000E0DD
:10149000B0919600B017B8F3F894E3D8E2D8E1D849
:1014A0007894D4D820928600B091BA00B33009F471
:1014B00073C0C4D8B091BE00B13008F46DC0B09113
:1014C0006A00B13008F468C085FD18C0B09196007C
:1014D000BF3F08F461C0F894CDD87894B5D8B091E6
:1014E0009600B130C0F7F894BCD8AAD8BAD878948E
:1014F000ABD8B0919600BF3FB0F3D2C2B3E09B2E01
:101500009068F894BEDE78949FD8F8949F77B9DEFF
:1015100080909600B0919600BF37789408F444C04C
:101520008BD8F894A7D878949A9451F7C7DEB82D41
:10153000B093C9008BD8F8941FD285D27894BAE0C2
:101540009B2E9068F8949DDE78947ED8F8949F77CF
:1015500098DE80909600B0919600BF37789478F727
:101560006BD8F8947ED86CD87CD878949A9449F744
:10157000A5DEB82DBB5FB093C80068D8F894FCD145
:1015800071D2789461D8F8947CDE7894B09196000A
:10159000BF3F08F499CF84C200919600B0918600B5
:1015A0000B1710F0009386004FD801E0B091BA00FD
:1015B000B35009F405E0B0919600B01708F074CF6D
:1015C000F89458D857D856D8789440D820926A00C2
:1015D00020926B0020926C00B0916B00B395B09399
:1015E0006B00BF3F71F5B0916C00B395B0936C0088
:1015F000B091CC0009E1BA9559F002E3BA9541F0F7
:101600000DE7BA9529F00AEFBA9511F020926C0017
:10161000B0916C00B017A8F094DD0ED8B0916C00BA
:10162000BA95B0936C0020926B00B091CB00B09350
:10163000AD00F8941FD87894B091CA00B093AD0073
:1016400003D8FED7B0916800BB2319F485FF01C011
:101650008FCE01E085FD01C006E0B0919600B01785
:1016600008F4BACFB091BA00B35009F0EDD7B091F9
:101670006800BB2309F47CCEF89463DD20926100FE
:101680002092620020926300522C209264002092EB
:10169000A1007894B091B700BB0FB0939F00209247
:1016A0007E0020927F002092800020928100209274
:1016B00082002092AA0060E070E020927100B8E001
:1016C000B093AA007061B8D7B2E074FDB1E0B7B9C9
:1016D000B6B1B068B064B6B9B6B1B6FDFDCF04B16D
:1016E00015B1B6B1BF77B6B9112309F00FEF00936A
:1016F000AB006CD9B8E0B093AA00706175DDF894C6
:10170000BFEFB0939B00C1D9B0916100B0939B0033
:10171000B0939C00B0939D007894B1E0B0936100C9
:10172000B09363005B2EB0936400B093A400B091BB
:101730009A00B093A300B091BA00B33019F49F7D22
:1017400087FD90627160726020926D00A3DCB9DC4D
:10175000B5D9BAD9B3D9B8D9B1D923DB08D8BDDB4B
:10176000EDDBB2D917DB66FD3BD877FFEDD877FD0F
:101770001BD9B3DBFADBA8D914DB66FD4DD8ADDB92
:1017800033DCA2D907DB66FD81D8A7DB44DC9CD91A
:1017900008DB66FDABD8A1DB7DDC96D9FBDAB2E0D5
:1017A00074FDB1E0B7B9B6B1B068B064B6B995DB55
:1017B00088DC8AD90BD971FF24C0B0919E00B09308
:1017C0009B00B0939C00B0919A00B093A300B1E04D
:1017D000B093A40018E12CE0B0916D00B11758F05F
:1017E0007D7F746020936F00B0919E00B0939B004A
:1017F000B0939D0006C0B0919600B13008F0ADCF17
:1018000060C072FF11C067FD0FC0B0916F00BA9544
:1018100019F47B7F7860A1CFB0936F00B0919600F0
:10182000B13008F09ACF4DC020927000B09199006D
:101830000AEF1091D600112309F003E0B01708F069
:1018400040C085FF04C0B0916800BB23D1F1B091C6
:10185000BA00B33081F495FD03C087FD04C00BC00E
:1018600087FF01C008C067FD06C06068B0919E0098
:10187000B0939B0087CF00EF67FF05C0B0919E003B
:10188000B0939B0000E2B0917B00B01708F465CFE5
:1018900067FF17C06F779F7D87FD90627460B2E12C
:1018A000B0936F00B0919E00B0939B0056CFB09163
:1018B0007000B395B0937000B0919600BB2309F00F
:1018C00002C020927000F8943CDC8090B900B2E035
:1018D000B093B90089DC8092B90020926100209217
:1018E000620020926300522C2092640020929F009C
:1018F00060E070E07894A8D624DC0091D600002344
:1019000019F0959AAC9AC09AB6B1B460B6B985FF91
:1019100005C0B0917000B43008F02ACD59CEEDE08A
:10192000F0E023D0053509F01BC0EEE0F0E01DD05B
:101930000A3A09F015C03AE0A2EBB0E0E3E0F0E0CB
:1019400014D00D9331963A95D9F739E1AEEBB0E06A
:10195000EFE0F0E00AD00D9331963A95D9F702C046
:10196000FDDB0AD0E8E2F0E00895E199FECFEEBB9E
:10197000FFBBE09A0DB308951ED03AE0A2EBB0E0B1
:10198000E3E0F0E00D910FD031963A95D9F739E1C7
:10199000AEEBB0E0EFE0F0E00D9105D031963A9576
:1019A000D9F712D00895E199FECF0DBBEEBBFFBB76
:1019B000E29AE19A0895EDE0F0E00FEFF4DFEEE057
:1019C000F0E00FEFF0DF0895EDE0F0E005E5EBDF8C
:1019D000EEE0F0E00AEAE7DF08953091AE00009112
:1019E000AF00313011F40093B200323011F40093A3
:1019F000B300333011F40093B400343011F4009389
:101A0000B600353011F40093B800363011F400936D
:101A1000C400373011F40093B900383011F400934A
:101A2000D500393011F40093CE003A3011F4009310
:101A3000BA003B3011F40093BB00089525E006D6B0
:101A40002A95E9F708950DD60FD611D613D6F8D5F5
:101A500008D60AD60CD60ED6F3D503D605D607D6A9
:101A600009D6089507D603D6FFD5FBD5E9D502D60A
:101A7000FED5FAD5F6D5E4D5FDD5F9D5F5D5F1D510
:101A800008958090AE009090AF00EBD5EAD5E9D5EF
:101A9000D7D58A94D1F7EED5D3D59A94E1F70895A6
:101AA000F894D1DF7894CADFC9DFB1E0B093AE001B
:101AB000B1E0B093AF002092B000F894E2DF7894E8
:101AC000B5E06B2E70909600C1D5B09196007B1654
:101AD000C9F7B13018F0BF3F40F107C07EDFF8947E
:101AE0004BDFB1DFB8E0B1BDA9DF6A9459F7B0911F
:101AF000B000B395B093B000B33008F4DECF9EDFF2
:101B0000B091AF00B395B093AF00F894B091AE0030
:101B1000BA95EEE3F0E0EB0FF21D04917894039593
:101B2000B091AF00B01708F4C6CF88DF87DFB0915F
:101B3000AE00B395B093AE00B091AE00BC3008F4E7
:101B4000B7CF0CDBF89418DFB8E0B1BD77DFCDCBB1
:00000001FF
